:020000040800F2
:1000000000060020E1010008E3010008E301000808
:10001000E3010008E3010008E3010008E301000830
:10002000E3010008E3010008E3010008B92F00081C
:10003000E3010008E3010008E3010008E301000810
:10004000E3010008E3010008E3010008E301000800
:10005000E3010008E301000861320008893200086A
:10006000B1320008D932000801330008E30100086A
:10007000E3010008E3010008E3010008E3010008D0
:10008000E3010008E3010008E3010008E3010008C0
:10009000E3010008E3010008E30100082933000838
:1000A000E3010008E3010008E3010008E3010008A0
:1000B000FD330008E3010008E3010008E301000844
:1000C000E3010008E3010008E3010008E301000880
:1000D000E3010008E3010008E3010008E301000870
:1000E0008D330008E3010008E3010008E301000884
:1000F000E3010008E3010008E3010008E301000850
:10010000E3010008E3010008E3010008E30100083F
:10011000E3010008E3010008E3010008E30100082F
:10012000E3010008E3010008E3010008E30100081F
:10013000E3010008E3010008E3010008E30100080F
:10014000E3010008E3010008E30100086D2700084F
:10015000E3010008E3010008E3010008E3010008EF
:10016000E3010008E3010008E3010008E3010008DF
:10017000E3010008E3010008E3010008E3010008CF
:10018000E3010008E3010008E3010008E3010008BF
:10019000E3010008E3010008E3010008E3010008AF
:1001A000E3010008E3010008E3010008E30100089F
:1001B000E3010008E3010008E3010008E30100088F
:1001C000E3010008E3010008E3010008E30100087F
:1001D000E3010008E3010008E3010008E30100086F
:1001E00002E000F000F8FEE772B6374880F30888B6
:1001F000364880F3098836483649086040F20000E6
:10020000CCF200004EF63471CEF200010860BFF36C
:100210004F8FBFF36F8F40F20000C0F2F0004EF638
:100220008851CEF200010860BFF34F8FBFF36F8F8C
:100230004FF00000E1EE100A4EF63C71CEF20001E4
:100240000860062080F31488BFF36F8F01F056FF1B
:1002500002F050FE4FF055301F491B4A91423CBFFF
:1002600041F8040BFAE71D49184A91423CBF41F896
:10027000040BFAE71A491B4A1B4B9A423EBF51F83E
:10028000040B42F8040BF8E700201849184A914281
:100290003CBF41F8040BFAE701F034FF02F07EFEA8
:1002A000144C154DAC4203DA54F8041B8847F9E7A7
:1002B00000F042F8114C124DAC4203DA54F8041B22
:1002C0008847F9E701F01CBF00060020002200204B
:1002D0000000000808ED00E00000002000060020FB
:1002E000C8370008002200204022002040220020C1
:1002F000602E0020E0010008E0010008E001000895
:10030000E00100082DE9F04F2DED108AC1F80CD066
:10031000C3689D46BDEC108ABDE8F08F002383F3CF
:1003200011882846A047002001F084FAFEE701F07A
:10033000EDF900DFFEE7000038B500F061FB01F0E9
:10034000ADFE054601F0D0FE0446D8B90F4B9D42E4
:100350001AD001339D4218BF044641F2883504BFCC
:1003600001240025002001F0A3FE0CB100F076F876
:1003700000F0ECFC00F09AFB284600F0B7F800F023
:100380006DF8F9E70025EDE70546EBE7010007B05A
:1003900008B500F05DFBA0F120035842584108BDAC
:1003A00007B541F21203022101A8ADF8043000F0B4
:1003B0006DFB03B05DF804FB38B5302383F311887F
:1003C000174803680BB101F001FB164A14480023DB
:1003D0004FF47A7101F0F0FA002383F31188124C84
:1003E000236813B12368013B2360636813B163681A
:1003F000013B63600D4D2B7833B963687BB90220F4
:1004000000F01EFC322363602B78032B07D1636856
:100410002BB9022000F014FC4FF47A73636038BDEE
:1004200040220020B9030008602300205822002049
:10043000084B187003280CD8DFE800F00805020804
:10044000022000F0F3BB022000F0E6BB024B0022CA
:100450005A60704758220020602300201F4B204A1A
:1004600010B51C461968013136D004339342F9D1D6
:100470006268A24230D31B4B9B6803F1006303F513
:1004800040439A4228D2002000F02AFB0220FFF7C6
:10049000CFFF154B1A6C00221A64196E1A66196E7A
:1004A000596C5A64596E5A665A6E1A6942F0005273
:1004B0001A611A6922F000521A611B6972B64FF074
:1004C000E0233021C3F8084DD4E9003281F31188CC
:1004D0009D4683F30888104710BD00BF00C0000888
:1004E00020C0000800220020003802402DE9F04F13
:1004F00093B0AA4B00902022FF210AA89D6800F02B
:10050000CFFBA74A1378A3B9A64801210360117055
:10051000302383F3118803680BB101F057FAA24A24
:10052000A04800234FF47A7101F046FA002383F3C8
:100530001188009B13B19D4B009A1A609C4A009C45
:100540001378032B1EBF00231370984A4FF0000A44
:1005500018BF5360D3465646D146012000F066FBD3
:1005600024B1924B1B68002B00F01182002000F098
:100570006FFA0390039B002BF2DB012000F04CFB91
:10058000039B213B162BE8D801A252F823F000BFB1
:10059000ED05000815060008A90600085B0500081F
:1005A0005B0500085B050008330700080309000825
:1005B0001D0800087F080008A7080008CD080008EB
:1005C0005B050008DF0800085B050008510900080A
:1005D0008D0600085B05000895090008F90500086C
:1005E0008D0600085B0500087F0800080220FFF761
:1005F000CFFE002840F0F581009B0221BAF1000FE8
:1006000008BF1C4605A841F21233ADF8143000F0C3
:100610003DFAA2E74FF47A7000F01AFA071EEBDBFE
:100620000220FFF7B5FE0028E6D0013F052F00F2BB
:10063000DA81DFE807F0030A0D101336052305936E
:10064000042105A800F022FA17E054480421F9E734
:1006500058480421F6E758480421F3E74FF01C08F6
:10066000404600F03FFA08F104080590042105A86F
:1006700000F00CFAB8F12C0FF2D1012000FA07F7C4
:1006800047EA0B0B5FFA8BFB4FF0000900F054FBBD
:1006900026B10BF00B030B2B08BF0024FFF780FEE5
:1006A0005BE746480421CDE7002EA5D00BF00B03F5
:1006B0000B2BA1D10220FFF76BFE074600289BD031
:1006C000012000F00DFA0220FFF7B2FE00261FFA0B
:1006D00086F8404600F014FA044690B100214046E6
:1006E00000F01EFA01360028F1D1BA46044641F264
:1006F0001213022105A8ADF814303E4600F0C6F9E9
:100700002BE70120FFF794FE2546244B9B68AB4264
:1007100007D9284600F0E6F9013040F0678104353A
:10072000F3E7234B00251D70204BBA465D603E4623
:10073000ACE7002E3FF460AF0BF00B030B2B7FF404
:100740005BAF0220FFF774FE322000F081F9B0F1B8
:100750000008FFF651AF18F003077FF44DAF0F4AC2
:10076000926808EB050393423FF646AFB8F5807FE9
:100770003FF742AF124B0193B84523DD4FF47A7037
:1007800000F066F90390039A002AFFF635AF019B4B
:10079000039A03F8012B0137EDE700BF0022002088
:1007A0005C23002040220020B903000860230020C1
:1007B0005822002004220020082200200C220020C1
:1007C0005C220020C820FFF7E3FD074600283FF425
:1007D00013AF1F2D11D8C5F1200242450AAB25F0F9
:1007E000030028BF424683490192184400F032FAC0
:1007F000019A8048FF2100F053FA4FEAA8037D498F
:100800000193C8F38702284600F052FA06460028F2
:100810003FF46DAF019B05EB830537E70220FFF73F
:10082000B7FD00283FF4E8AE00F0A6F900283FF439
:10083000E3AE0027B846704B9B68BB4218D91F2F08
:1008400011D80A9B01330ED027F0030312AA1344D8
:1008500053F8203C05934046042205A900F0A0FA75
:1008600004378046E7E7384600F03CF90590F2E7A8
:10087000CDF81480042105A800F008F906E700234C
:10088000642104A8049300F0F7F800287FF4B4AEC4
:100890000220FFF77DFD00283FF4AEAE049800F083
:1008A00053F90590E6E70023642104A8049300F0BF
:1008B000E3F800287FF4A0AE0220FFF769FD0028CE
:1008C0003FF49AAE049800F04FF9EAE70220FFF7F0
:1008D0005FFD00283FF490AE00F05EF9E1E70220F2
:1008E000FFF756FD00283FF487AE05A9142000F05D
:1008F00059F904210746049004A800F0C7F83946C6
:10090000B9E7322000F0A4F8071EFFF675AEBB076A
:100910007FF472AE384A926807EB090393423FF6C0
:100920006BAE0220FFF734FD00283FF465AE27F0E0
:1009300003074F44B9453FF4A9AE484600F0D2F84A
:100940000421059005A800F0A1F809F10409F1E7D8
:100950004FF47A70FFF71CFD00283FF44DAE00F015
:100960000BF9002844D00A9B01330BD008220AA9B6
:10097000002000F09DF900283AD02022FF210AA88B
:1009800000F08EF9FFF70CFD1C4800F059FF13B082
:10099000BDE8F08F002E3FF42FAE0BF00B030B2BB6
:1009A0007FF42AAE0023642105A8059300F064F8C3
:1009B000074600287FF420AE0220FFF7E9FC8046BE
:1009C00000283FF419AEFFF7EBFC41F2883000F04D
:1009D00037FF059800F0E2F9464600F0ADF93C46D5
:1009E000BBE5064652E64FF0000905E6BA467EE64C
:1009F00037467CE65C22002000220020A086010011
:100A00007047000070B50F4B1B780133DBB2012B30
:100A10000C4611D80C4D29684FF47A730E6AA2FB6C
:100A20000332014622462846B047844204D1074B90
:100A300000221A70012070BD4FF4FA7000F000FF20
:100A40000020F8E710220020082600209423002030
:100A500007B50023024601210DF107008DF807308C
:100A6000FFF7D0FF20B19DF8070003B05DF804FB4D
:100A70004FF0FF30F9E700000A4608B50421FFF700
:100A8000C1FF80F00100C0B2404208BD30B4054C47
:100A90002368DD69044B0A46AC460146204630BC5B
:100AA000604700BF08260020A086010070B501F055
:100AB000E7F9094E094D30800024286833888342C5
:100AC00008D901F0D7F92B6804440133B4F5404F3D
:100AD0002B60F2D370BD00BF962300206823002056
:100AE00001F090BA00F1006000F5404000687047E6
:100AF00000F10060920000F5404001F00FBA0000E4
:100B0000054B1A68054B1B889B1A834202D9104477
:100B100001F0B0B900207047682300209623002020
:100B200038B5084D044629B128682044BDE838404E
:100B300001F0C0B92868204401F0A4F90028F3D0DE
:100B400038BD00BF6823002010F003030AD1B0F5C0
:100B5000047F05D200F10050A0F51040D0F8003815
:100B6000184670470023FBE700F10050A0F5104045
:100B7000D0F8100A70470000064991F8243033B1CC
:100B80000023086A81F824300822FFF7B1BF012052
:100B9000704700BF6C230020014B1868704700BFEE
:100BA000002004E070B5194B1D68194B0138C5F3DE
:100BB0000B0408442D0C04221E88A6420BD15C684D
:100BC0000A46013C824213460FD214F9016F4EB11E
:100BD00002F8016BF6E7013A03F10803ECD1814218
:100BE0000B4602D22C2203F8012B0A4A0524168850
:100BF000AE4204D1984284BF967803F8016B013C61
:100C000002F10402F3D1581A70BD00BF002004E0C5
:100C1000E0340008CC340008022802BF024B4FF039
:100C200080729A61704700BF00000240022802BF34
:100C3000024B4FF480729A61704700BF000002407F
:100C4000022801BF024A536983F4807353617047DD
:100C50000000024010B50023934203D0CC5CC45482
:100C60000133F9E710BD000010B5013810F9013F5C
:100C70003BB191F900409C4203D11AB10131013AD4
:100C8000F4E71AB191F90020981A10BD1046FCE75C
:100C900003460246D01A12F9011B0029FAD1704707
:100CA00002440346934202D003F8011BFAE770475F
:100CB0002DE9F8431F4D144695F824200746884631
:100CC00052BBDFF870909CB395F824302BB92022EA
:100CD000FF2148462F62FFF7E3FF95F82400C0F19B
:100CE0000802A24228BF2246D6B24146920005EB36
:100CF0008000FFF7AFFF95F82430A41B1E44F6B226
:100D0000082E17449044E4B285F82460DBD1FFF745
:100D100033FF0028D7D108E02B6A03EB820383421C
:100D2000CFD0FFF729FF0028CBD10020BDE8F88302
:100D30000120FBE76C230020024B1A78024B1A704B
:100D4000704700BF942300201022002010B50F4CE4
:100D50000F4800F0B5F821460D4800F0DDF8246892
:100D60000C48626DD2F8043843F00203C2F804382C
:100D700000F066FD0849204600F0D4F9626DD2F813
:100D8000043823F00203C2F8043810BDAC35000863
:100D90000826002040420F00B435000870470000CC
:100DA00030B5094D0A4491420DD011F8013B58402D
:100DB000082340F30004013B2C4013F0FF0384EAB6
:100DC0005000F6D1EFE730BD2083B8ED02684368EC
:100DD0001143016003B118477047000013B5446B1D
:100DE000D4F894341A681178042915D1217C022989
:100DF00012D11979128901238B4013420CD101A918
:100E000004F14C0001F032FFD4F89444019B2179A5
:100E10000246206800F0D0F902B010BD143001F095
:100E2000B5BE00004FF0FF33143001F0AFBE00003C
:100E30004C3001F087BF00004FF0FF334C3001F021
:100E400081BF0000143001F083BE00004FF0FF317D
:100E5000143001F07DBE00004C3001F053BF0000A3
:100E60004FF0FF324C3001F04DBF000000207047C2
:100E700010B5D0F894341A6811780429044617D1B3
:100E8000017C022914D15979528901238B401342E4
:100E90000ED1143001F016FE024648B1D4F8944445
:100EA0004FF4807361792068BDE8104000F072B99A
:100EB00010BD0000406BFFF7DBBF00007047000073
:100EC0007FB5124B036000234360C0E90233012564
:100ED00002260F4B057404460290019300F1840230
:100EE000294600964FF48073143001F0C7FD094B7A
:100EF0000294CDE9006304F523724FF48073294610
:100F000004F14C0001F08EFE04B070BD0035000805
:100F1000B50E0008DD0D00080B68302282F3118841
:100F20000A7903EB820290614A79093243F8220080
:100F30008A7912B103EB820398610223C0F89414FA
:100F40000374002080F311887047000038B5037FD8
:100F5000044613B190F85430ABB9201D012502218D
:100F6000FFF734FF04F1140025776FF0010100F062
:100F70008FFC84F8545004F14C006FF00101BDE87F
:100F8000384000F085BC38BD10B50121044604305E
:100F9000FFF71CFF0023237784F8543010BD0000B6
:100FA00038B504460025143001F080FD04F14C00F2
:100FB000257701F04FFE201D84F854500121FFF7E2
:100FC00005FF2046BDE83840FFF752BF90F8443097
:100FD00003F06003202B07D190F84520212A4FF021
:100FE000000303D81F2A06D800207047222AFBD10D
:100FF000C0E90E3303E0034A82630722C26303643D
:10100000012070471122002037B5D0F894341A68B7
:101010001178042904461AD1017C022917D11979C3
:10102000128901238B40134211D100F14C0528464F
:1010300001F0D0FE58B101A9284601F017FED4F8FE
:101040009444019B21790246206800F0B5F803B072
:1010500030BD0000F0B500EB810385B09E69044609
:101060000D46FEB1302383F3118804EB8507301D54
:101070000821FFF7ABFEFB685B691B6806F14C00BB
:101080001BB1019001F000FE019803A901F0EEFDF3
:10109000024648B1039B2946204600F08DF8002304
:1010A00083F3118805B0F0BDFB685A691268002A05
:1010B000F5D01B8A013B1340F1D104F14402EAE769
:1010C000093138B550F82140DCB1302383F3118861
:1010D000D4F894241368527903EB8203DB689B698C
:1010E0005D6845B104216018FFF770FE294604F1E0
:1010F000140001F0F1FC2046FFF7BAFE002383F351
:10110000118838BD7047000001F050B8012303700A
:101110000023C0E90133C36183620362C362436297
:101120000363704738B50446302383F311880025E4
:10113000C0E90355C0E90555416001F047F80223B5
:10114000237085F31188284638BD000070B500EB88
:10115000810305465069DA600E46144618B1102224
:101160000021FFF79DFDA06918B110220021FFF7B3
:1011700097FD31462846BDE8704001F0F1B8000007
:10118000826802F0011282600022C0E904228261BA
:1011900001F072B9F0B400EB81044789E4680125DD
:1011A000A4698D403D43458123600023A2606360B4
:1011B000F0BC01F08DB90000F0B400EB81040789A8
:1011C000E468012564698D403D4305812360002367
:1011D000A2606360F0BC01F007BA000070B50223A2
:1011E000002504460370C0E90255C0E90455C564F2
:1011F000856180F8345001F04FF863681B6823B1B3
:1012000029462046BDE87040184770BD0378052B7D
:1012100010B504460AD080F85030052303704368A7
:101220001B680BB1042198470023A36010BD000088
:101230000178052906D190F85020436802701B6898
:1012400003B118477047000070B590F83430044679
:1012500013B1002380F8343004F14402204601F039
:101260002DF963689B68B3B994F8443013F06005B6
:1012700035D00021204601F0CDFB0021204601F0B1
:10128000BFFB63681B6813B10621204698470623FD
:1012900084F8343070BD204698470028E4D0B4F874
:1012A0004A30E26B9A4288BFE36394F94430E56BBD
:1012B000002B4FF0300380F20381002D00F0F2800C
:1012C000092284F8342083F311880021D4E90E2305
:1012D0002046FFF771FF002383F31188DAE794F8C3
:1012E000452003F07F0343EA022340F20232934297
:1012F00000F0C58021D8B3F5807F48D00DD8012BF0
:101300003FD0022B00F09380002BB2D104F14C02AD
:10131000A2630222E2632364C1E7B3F5817F00F098
:101320009B80B3F5407FA4D194F84630012BA0D127
:10133000B4F84C3043F0020332E0B3F5006F4DD007
:1013400017D8B3F5A06F31D0A3F5C063012B90D8A7
:10135000636894F846205E6894F84710B4F8483003
:101360002046B047002884D04368A3630368E36342
:101370001AE0B3F5106F36D040F6024293427FF484
:1013800078AF5C4BA3630223E3630023C3E794F8C5
:101390004630012B7FF46DAFB4F84C3023F00203DC
:1013A000C4E90E55A4F84C30256478E7B4F844300D
:1013B000B3F5A06F0ED194F8463084F84E30204635
:1013C00000F0C2FF63681B6813B1012120469847F3
:1013D000032323700023C4E90E339CE704F14F0379
:1013E000A3630123C3E72378042B10D1302383F3B5
:1013F00011882046FFF7C4FE85F311880321636836
:1014000084F84F5021701B680BB12046984794F820
:101410004630002BDED084F84F30042323706368FD
:101420001B68002BD6D0022120469847D2E794F8BB
:1014300048301D0603F00F0120460AD501F030F8B0
:10144000012804D002287FF414AF2B4B9AE72B4BD2
:1014500098E701F017F8F3E794F84630002B7FF493
:1014600008AF94F8483013F00F01B3D01A062046A5
:1014700002D501F0E3FAADE701F0D6FAAAE794F855
:101480004630002B7FF4F5AE94F8483013F00F018E
:10149000A0D01B06204602D501F0BCFA9AE701F065
:1014A000AFFA97E7142284F8342083F311882B468F
:1014B0002A4629462046FFF76DFE85F31188E9E6A6
:1014C0005DB1152284F8342083F311880021D4E91A
:1014D0000E232046FFF75EFEFDE60B2284F8342043
:1014E00083F311882B462A4629462046FFF764FEDF
:1014F000E3E700BF30350008283500082C35000828
:1015000038B590F834300446002B3ED0063BDAB2B2
:101510000F2A34D80F2B32D8DFE803F037313108E7
:10152000223231313131313131313737C56BB0F899
:101530004A309D4214D2C3681B8AB5FBF3F203FB09
:1015400012556DB9302383F311882B462A4629465C
:10155000FFF732FE85F311880A2384F834300EE059
:10156000142384F83430302383F3118800231A467F
:1015700019462046FFF70EFE002383F3118838BD7D
:10158000036C03B198470023E7E70021204601F0F0
:1015900041FA0021204601F033FA63681B6813B159
:1015A0000621204698470623D7E7000010B590F89B
:1015B0003430142B044629D017D8062B05D001D877
:1015C0001BB110BD093B022BFBD80021204601F0C6
:1015D00021FA0021204601F013FA63681B6813B159
:1015E000062120469847062319E0152BE9D10B2345
:1015F00080F83430302383F3118800231A461946CB
:10160000FFF7DAFD002383F31188DAE7C3689B69EB
:101610005B68002BD5D1036C03B19847002384F895
:101620003430CEE700230375826803691B6899682C
:101630009142FBD25A680360426010605860704764
:1016400000230375826803691B6899689142FBD87F
:101650005A680360426010605860704708B50846D9
:10166000302383F311880B7D032B05D0042B0DD081
:101670002BB983F3118808BD8B6900221A604FF0E3
:10168000FF338361FFF7CEFF0023F2E7D1E9003299
:1016900013605A60F3E70000FFF7C4BF054BD96839
:1016A0000875186802681A60536001220275D860D4
:1016B000FEF728BE9823002030B50C4BDD684B1C8C
:1016C00087B004460FD02B46094A684600F074F9EB
:1016D0002046FFF7E3FF009B13B1684600F076F960
:1016E000A86907B030BDFFF7D9FFF9E798230020BC
:1016F0005D160008044B1A68DB6890689B68984286
:1017000094BF00200120704798230020084B10B59B
:101710001C68D86822681A60536001222275DC6058
:10172000FFF78EFF01462046BDE81040FEF7EABDF8
:1017300098230020044B1A68DB6892689B689A42E1
:1017400001D9FFF7E3BF70479823002038B5074C55
:1017500007490848012300252370656001F072FBEA
:101760000223237085F3118838BD00BF00260020B6
:10177000383500089823002000F05EB9EFF311809F
:1017800020B9EFF30583302282F3118870470000FF
:1017900010B530B9EFF30584C4F3080414B180F335
:1017A000118810BDFFF7C6FF84F31188F9E7000028
:1017B000034A516853685B1A9842FBD8704700BFD0
:1017C000001000E08B60022308618B82084670479E
:1017D0008368A3F1840243F8142C026943F8442C73
:1017E000426943F8402C094A43F8242CC26843F864
:1017F000182C022203F80C2C002203F80B2C044AAC
:1018000043F8102CA3F12000704700BF1D0300080F
:101810009823002008B5FFF7DBFFBDE80840FFF77D
:101820003BBF0000024BDB6898610F20FFF736BF1B
:1018300098230020302383F31188FFF7F3BF0000C3
:1018400008B50146302383F311880820FFF734FFE1
:10185000002383F3118808BD064BDB6839B1426869
:1018600018605A60136043600420FFF725BF4FF0F3
:10187000FF307047982300200368984206D01A680A
:101880000260506099611846FFF706BF704700007C
:1018900038B504460D462068844200D138BD03683F
:1018A00023605C608561FFF7F7FEF4E710B503681D
:1018B0009C68A2420CD85C688A600B604C60216016
:1018C000596099688A1A9A604FF0FF33836010BD9F
:1018D0001B68121BECE700000A2938BF0A2170B50B
:1018E00004460D460A26601901F0A6FA01F092FAA4
:1018F000041BA54203D8751C2E460446F3E70A2EA6
:1019000004D9BDE87040012001F0DCBA70BD0000D0
:10191000F8B5144B0D46D96103F1100141600A2A54
:101920001969826038BF0A22016048601861A818EE
:10193000144601F073FA0A2701F06CFA431BA34224
:10194000064606D37C1C281901F076FA2746354650
:10195000F2E70A2F04D9BDE8F840012001F0B2BA3D
:10196000F8BD00BF98230020F8B506460D4601F0EB
:1019700051FA0F4A134653F8107F9F4206D12A4668
:1019800001463046BDE8F840FFF7C2BFD169BB68E9
:10199000441A2C1928BF2C46A34202D92946FFF726
:1019A0009BFF224631460348BDE8F840FFF77EBF63
:1019B00098230020A823002010B4C0E903230023AB
:1019C0005DF8044B4361FFF7CFBF000010B5194C21
:1019D000236998420DD0D0E90032816813605A60C3
:1019E0009A680A449A60002303604FF0FF33A361B2
:1019F00010BD2346026843F8102F53600022026096
:101A000022699A4203D1BDE8104001F00FBA9368F1
:101A100081680B44936001F0FDF92269E1699268E5
:101A2000441AA242E4D91144BDE81040091AFFF754
:101A300053BF00BF982300202DE9F047DFF8BC809A
:101A400008F110072C4ED8F8105001F0E3F9D8F83F
:101A50001C40AA68031B9A423ED81444D5E90032C0
:101A60004FF00009C8F81C4013605A60C5F8009098
:101A7000D8F81030B34201D101F0D8F989F31188B8
:101A8000D5E9033128469847302383F311886B69E1
:101A9000002BD8D001F0BEF96A69A0EB04094A45D1
:101AA00082460DD2022001F00DFA0022D8F8103043
:101AB000B34208D151462846BDE8F047FFF728BF9A
:101AC000121A2244F2E712EB090938BF4A462946A6
:101AD0003846FFF7EBFEB5E7D8F81030B34208D030
:101AE0001444211AC8F81C00A960BDE8F047FFF7AC
:101AF000F3BEBDE8F08700BFA82300209823002094
:101B000000207047FEE70000704700004FF0FF30F4
:101B10007047000002290CD0032904D0012907488E
:101B200018BF00207047032A05D8054800EBC20003
:101B30007047044870470020704700BF1036000807
:101B400020220020C435000870B59AB0054608462A
:101B500001A9144600F0C2F801A8FFF799F8431C48
:101B60005B00C5E900340022237003236370C6B212
:101B700001AB02341046D1B28E4204F1020401D806
:101B80001AB070BD13F8011B04F8021C04F8010C14
:101B90000132F0E708B5302383F311880348FFF7DB
:101BA00033FA002383F3118808BD00BF0826002004
:101BB00090F8443003F01F02012A07D190F8452025
:101BC0000B2A03D10023C0E90E3315E003F06003B4
:101BD000202B08D1B0F848302BB990F84520212AA5
:101BE00003D81F2A04D8FFF7F1B9222AEBD0FAE76D
:101BF000034A82630722C26303640120704700BF67
:101C00001822002007B5052917D8DFE801F01916BA
:101C100003191920302383F31188104A0190012100
:101C2000FFF794FA01980E4A0221FFF78FFA0D4848
:101C3000FFF7B6F9002383F3118803B05DF804FBC6
:101C4000302383F311880748FFF780F9F2E7302348
:101C500083F311880348FFF797F9EBE76435000831
:101C6000883500080826002038B50C4D0C4C0D496D
:101C70002A4604F10800FFF767FF05F1CA0204F1E4
:101C800010000949FFF760FF05F5CA7204F118005A
:101C90000649BDE83840FFF757BF00BFD02A0020F3
:101CA00020220020443500084E3500085935000830
:101CB00070B5044608460D46FEF7EAFFC6B2204658
:101CC000013403780BB9184670BD32462946FEF739
:101CD000CBFF0028F3D10120F6E700002DE9F04703
:101CE00005460C46FEF7D4FF2B49C6B22846FFF73F
:101CF000DFFF08B10A36F6B228492846FFF7D8FFB9
:101D000008B11036F6B2632E0BD8DFF88C80DFF8FE
:101D10008C90234FDFF894A02E7846B92670BDE84A
:101D2000F08729462046BDE8F04701F0B1BB252EDB
:101D30002ED1072241462846FEF796FF70B9194B6F
:101D4000224603F1100153F8040B42F8040B8B42B6
:101D5000F9D11B78137007351134DDE708224946A5
:101D60002846FEF781FF98B90F4BA21C1978090984
:101D70000232C95D02F8041C13F8011B01F00F01C7
:101D80005345C95D02F8031CF0D118340835C3E788
:101D900004F8016B0135BFE73036000859350008FB
:101DA0004A36000838360008107AFF1F1C7AFF1FD9
:101DB000BFF34F8F024AD368DB03FCD4704700BFE8
:101DC000003C024008B5094B1B7873B9FFF7F0FFE0
:101DD000074B1A69002ABFBF064A5A6002F18832CF
:101DE0005A601A6822F480621A6008BD2E2D002005
:101DF000003C02402301674508B50B4B1B7893B9A3
:101E0000FFF7D6FF094B1A6942F000421A611A68BF
:101E100042F480521A601A6822F480521A601A68DA
:101E200042F480621A6008BD2E2D0020003C024062
:101E30000B28F0B516D80C4C0C4923787BB90C4D07
:101E40000E460C234FF0006255F8047B46F8042B35
:101E5000013B13F0FF033A44F6D10123237051F8FC
:101E60002000F0BD0020FCE7602D0020302D002078
:101E70005C360008014B53F8200070475C360008C0
:101E80000C2070470B2810B5044601D9002010BD66
:101E9000FFF7CEFF064B53F824301844C21A0BB993
:101EA0000120F4E712680132F0D1043BF6E700BFED
:101EB0005C3600080B2838B5044628D8FFF75EFCCE
:101EC000FFF776FFFFF77EFF124AF323D360E300AC
:101ED000DBB243F4007343F002031361136943F46C
:101EE0008033136105462046FFF762FFFFF7A0FF2E
:101EF000094B53F8241000F0E9F82846FFF77CFF5F
:101F0000FFF746FC2046BDE83840FFF7BBBF002086
:101F100038BD00BF003C02405C36000812F00103EF
:101F20002DE9F04105460E4614464BD18218B2F118
:101F3000016F61D8314B1B6813F001035CD0304F47
:101F4000FFF71CFCFFF73EFFF323FB60FFF730FFBA
:101F5000314640F20128032C18D824F00104284E01
:101F60000C446D1A40F20118A142336905EB0107D8
:101F70002AD123F001033361FFF73EFFFFF708FC8E
:101F80000120BDE8F081043C0435E4E7AB07E4D16F
:101F90003B6923F440733B613B6943EA08033B61BF
:101FA00051F8046B2E60BFF34F8FFFF701FF2B68D2
:101FB0009E42E8D03B6923F001033B61FFF71CFF21
:101FC000FFF7E6FB0020DCE723F44073336133695D
:101FD00043EA080333610B883B80BFF34F8FFFF761
:101FE000E7FE3F8831F8023BBFB2BB42BCD0336949
:101FF00023F001033361E1E71846C2E700380240ED
:10200000003C0240084908B50B7828B11BB9FFF71E
:10201000D9FE01230B7008BD002BFCD0BDE80840A1
:102020000870FFF7E9BE00BF2E2D002010B5024456
:10203000064BD2B2904200D110BD441C00B253F8FE
:10204000200041F8040BE0B2F4E700BF5028004044
:102050000F4B30B51C6F240407D41C6F44F400747C
:102060001C671C6F44F400441C670A4C236843F44B
:10207000807323600244084BD2B2904200D130BD3D
:10208000441C00B251F8045B43F82050E0B2F4E77E
:1020900000380240007000405028004007B501227F
:1020A00001A90020FFF7C2FF019803B05DF804FB0F
:1020B00013B50446FFF7F2FFA04205D0012201A9A3
:1020C00000200194FFF7C4FF02B010BD704700006C
:1020D000034B1A681AB9034AD2F874281A60704779
:1020E000642D00200030024008B5FFF7F1FF024BDD
:1020F0001868C0F3407008BD642D002070470000D0
:10210000FEE700000A4B0B480B4A90420BD30B4BE7
:10211000DA1C121AC11E22F003028B4238BF0022C1
:102120000021FEF7BDBD53F8041B40F8041BECE78B
:1021300008380008602E0020602E0020602E00204D
:1021400070B5D0E915439E6800224FF0FF3504EBCF
:1021500042135101D3F800090028BEBFD3F800098B
:1021600040F08040C3F80009D3F8000B0028BEBF40
:10217000D3F8000B40F08040C3F8000B0132631825
:102180009642C3F80859C3F8085BE0D24FF0011338
:10219000C4F81C3870BD0000890141F020010161C4
:1021A00003699B06FCD41220FFF702BB10B5054C57
:1021B0002046FEF7ABFF4FF0A0436365024BA365DB
:1021C00010BD00BF682D0020B036000870B5037840
:1021D000012B054650D12A4B446D98421BD1294B07
:1021E0005A6B42F080025A635A6D42F080025A657F
:1021F0005A6D5A6942F080025A615A6922F080028F
:102200005A610E2143205B6900F022FC1E4BE36003
:102210001E4BC4F800380023C4F8003EC0232360DE
:102220006E6D4FF40413A3633369002BFCDA0123B2
:1022300033610C20FFF7BCFA3369DB07FCD41220B2
:10224000FFF7B6FA3369002BFCDA0026A6602846B1
:10225000FFF776FF6B68C4F81068DB68C4F8146891
:10226000C4F81C684BB90A4BA3614FF0FF3363619C
:10227000A36843F00103A36070BD064BF4E700BF01
:10228000682D002000380240401400400300200266
:10229000003C30C0083C30C0F8B5446D0546002114
:1022A0002046FFF779FFA96D00234FF001128F68D8
:1022B000C4F834384FF00066C4F81C284FF0FF30E3
:1022C00004EB431201339F42C2F80069C2F8006B6D
:1022D000C2F80809C2F8080BF2D20B686A6DEB6508
:1022E000636210231361166916F01006FBD11220E9
:1022F000FFF75EFAD4F8003823F4FE63C4F8003820
:10230000A36943F4402343F01003A3610923C4F8F5
:102310001038C4F814380A4BEB604FF0C043C4F8CF
:10232000103B084BC4F8003BC4F81069C4F80039EE
:10233000EB6D03F1100243F48013EA65A362F8BD6C
:102340008C36000840800010426D90F84E10D2F894
:10235000003823F4FE6343EA0113C2F800387047E3
:102360002DE9F84300EB8103456DDA68166806F045
:102370000306731E022B05EB41130C4680460FFA31
:1023800081F94FEA41104FF00001C3F8101B4FF0E4
:10239000010104F1100398BFB60401FA03F3916937
:1023A0008EBF334E06F1805606F5004600293AD01E
:1023B000578A04F15801490137436F50D5F81C186A
:1023C0000B43C5F81C382B180021C3F810195369AA
:1023D0000127611EA7409BB3138A928B9B08012A99
:1023E00088BF5343D8F85C20981842EA034301F1B0
:1023F000400205EB8202C8F85C0021465360284683
:10240000FFF7CAFE08EB8900C3681B8A43EA8453BE
:10241000483464011E432E51D5F81C381F43C5F8BB
:102420001C78BDE8F88305EB4917D7F8001B21F4A9
:102430000041C7F8001BD5F81C1821EA0303C0E7C8
:1024400004F13F0305EB83030A4A5A6028462146FC
:10245000FFF7A2FE05EB4910D0F8003923F4004342
:10246000C0F80039D5F81C3823EA0707D7E700BFC2
:102470000080001000040002826D1268C265FFF740
:102480005FBE00005831436D49015B5813F40040B2
:1024900004D013F4001F0CBF02200120704700007D
:1024A0004831436D49015B5813F4004004D013F4E4
:1024B000001F0CBF022001207047000000EB8101CB
:1024C000CB68196A0B6813604B6853607047000053
:1024D00000EB810330B5DD68AA691368D36019B9D0
:1024E000402B84BF402313606B8A1468426D1C44E8
:1024F000013CB4FBF3F46343033323F0030302EB27
:10250000411043EAC44343F0C043C0F8103B2B687A
:1025100003F00303012B09B20ED1D2F8083802EB05
:10252000411013F4807FD0F8003B14BF43F0805378
:1025300043F00053C0F8003B02EB4112D2F8003BDD
:1025400043F00443C2F8003B30BD00002DE9F041E8
:10255000244D6E6D06EB40130446D3F8087BC3F898
:10256000087B38070AD5D6F81438190706D505EBC5
:1025700084032146DB6828465B689847FA071FD525
:10258000D6F81438DB071BD505EB8403D968CCB922
:102590008B69488A5A68B2FBF0F600FB16228AB9AA
:1025A0001868DA6890420DD2121AC3E90024302369
:1025B00083F311880B482146FFF78AFF84F31188C3
:1025C000BDE8F081012303FA04F26B8923EA0203D8
:1025D0006B81CB68002BF3D021460248BDE8F04167
:1025E000184700BF682D002000EB810370B5DD683F
:1025F000436D6C692668E6604A0156BB1A444FF485
:102600000020C2F810092A6802F00302012A0AB267
:102610000ED1D3F8080803EB421410F4807FD4F8ED
:10262000000914BF40F0805040F00050C4F8000989
:1026300003EB4212D2F8000940F00440C2F800094E
:10264000D3F83408012202FA01F10143C3F8341827
:1026500070BD19B9402E84BF4020206020682E8AAA
:102660008419013CB4FBF6F440EAC44040F0005049
:102670001A44C6E72DE9F8433B4D6E6D06EB401357
:102680000446D3F80889C3F8088918F0010F4FEA07
:1026900040171AD0D6F81038DB0716D505EB8003A3
:1026A000D9684B691868DA68904230D2121A4FF034
:1026B00000091A60C3F80490302383F3118821467F
:1026C0002846FFF791FF89F3118818F0800F1CD07E
:1026D000D6F834380126A640334216D005EB8403E1
:1026E0006D6DD3F80CC0DCF814200134E4B2D2F8DC
:1026F00000E005EB04342F445168714515D3D5F83B
:10270000343823EA0606C5F83468BDE8F8830123A7
:1027100003FA04F22B8923EA02032B818B68002B36
:10272000D3D0214628469847CFE7BCF81000AEEB3F
:102730000103834228BF0346D7F8180980B2B3EBE0
:10274000800FE2D89068A0F1040959F8048FC4F80A
:102750000080A0EB09089844B8F1040FF5D818449C
:102760000B4490605360C7E7682D00202DE9F74FB8
:10277000A24C656D6E69AB691E4016F480586E619F
:1027800007D02046FEF72AFD03B0BDE8F04F00F069
:1027900047BC002E12DAD5F8003E98489B071EBFB2
:1027A000D5F8003E23F00303C5F8003ED5F8043801
:1027B00023F00103C5F80438FEF73AFD370505D5C7
:1027C0008E48FFF7BDFC8D48FEF720FDB0040CD508
:1027D000D5F8083813F0060FEB6823F470530CBFDC
:1027E00043F4105343F4A053EB6031071BD56368E7
:1027F000DB681BB9AB6923F00803AB612378052BB9
:102800000CD1D5F8003E7D489A071EBFD5F8003E92
:1028100023F00303C5F8003EFEF70AFD6368DB689A
:102820000BB176489847F30274D4B70227D5D4F891
:102830005490DFF8C8B100274FF0010A09EB4712A6
:10284000D2F8003B03F44023B3F5802F11D1D2F826
:10285000003B002B0DDA62890AFA07F322EA030330
:10286000638104EB8703DB68DB6813B139465846A4
:102870009847A36D01379B68FFB29F42DED9F006EF
:1028800017D5676D3A6AC2F30A1002F00F0302F41B
:10289000F012B2F5802F00F08580B2F5402F08D1FC
:1028A00004EB83030022DB681B6A07F58057904224
:1028B0006AD13003D5F8184813D5E10302D50020BA
:1028C000FFF744FEA20302D50120FFF73FFE63039A
:1028D00002D50220FFF73AFE270302D50320FFF7B7
:1028E00035FE75037FF550AFE00702D50020FFF7F6
:1028F000C1FEA10702D50120FFF7BCFE620702D589
:102900000220FFF7B7FE23077FF53EAF0320FFF756
:10291000B1FE39E7636DDFF8E4A0019300274FF0C3
:102920000109A36D9B685FFA87FB9B453FF67DAF6E
:10293000019B03EB4B13D3F8001901F44021B1F5CF
:10294000802F1FD1D3F8001900291BDAD3F8001902
:1029500041F09041C3F80019D3F800190029FBDBBE
:102960005946606DFFF718FC218909FA0BF321EA3B
:102970000303238104EB8B03DB689B6813B1594687
:10298000504698470137CCE7910708BFD7F8008039
:10299000072A98BF03F8018B02F1010298BF4FEAA2
:1029A000182884E7023304EB830207F58057526846
:1029B000D2F818C0DCF80820DCE9001CA1EB0C0CF4
:1029C000002188420AD104EB830463689B699A68FA
:1029D00002449A605A6802445A606AE711F0030F91
:1029E00008BFD7F800808C4588BF02F8018B01F141
:1029F000010188BF4FEA1828E3E700BF682D0020D7
:102A0000436D03EB4111D1F8003B43F40013C1F8CF
:102A1000003B7047436D03EB4111D1F8003943F49B
:102A20000013C1F800397047436D03EB4111D1F831
:102A3000003B23F40013C1F8003B7047436D03EBE8
:102A40004111D1F8003923F40013C1F8003970475F
:102A500000F1604303F561430901C9B283F8001333
:102A6000012200F01F039A4043099B0003F16043D9
:102A700003F56143C3F880211A60704730B5039CA9
:102A80000172043304FB0325C0E90653049B03636E
:102A90000021059BC160C0E90000C0E90422C0E933
:102AA0000842C0E90A11436330BD0000416A0022B8
:102AB000C0E90411C0E90A22C2606FF00101FEF70B
:102AC000E7BE0000D0E90432934201D1C2680AB9DE
:102AD000181D70470020704703691960C2680132F1
:102AE000C260C269134482690361934224BF436A8E
:102AF00003610021FEF7C0BE38B504460D46E36809
:102B00003BB16269131D1268A3621344E3620020A3
:102B100007E0237A33B929462046FEF79DFE0028B8
:102B2000EDDA38BD6FF00100FBE70000C368C26951
:102B3000013BC3604369134482694361934224BFEC
:102B4000436A436100238362036B03B118477047F4
:102B500070B53023044683F31188866A3EB9FFF7C7
:102B6000CBFF054618B186F31188284670BDA36ACD
:102B7000E26A13F8015BA362934202D32046FFF797
:102B8000D5FF002383F31188EFE700002DE9F84F0C
:102B900004460E46174698464FF0300989F31188CF
:102BA0000025AA46D4F828B0BBF1000F09D1414650
:102BB0002046FFF7A1FF20B18BF311882846BDE81E
:102BC000F88FD4E90A12A7EB050B521A934528BFD8
:102BD0009346BBF1400F1BD9334601F1400251F837
:102BE000040B43F8040B9142F9D1A36A40334036F9
:102BF000A3624035D4E90A239A4202D32046FFF764
:102C000095FF8AF31188BD42D8D289F31188C9E7AC
:102C100030465A46FEF71EF8A36A5B445E44A36240
:102C20005D44E7E710B5029C0172043303FB042105
:102C3000C0E906130023C0E90A33039B0363049B26
:102C4000C460C0E90000C0E90422C0E9084243634F
:102C500010BD0000026AC260426AC0E9042200227C
:102C6000C0E90A226FF00101FEF712BED0E9042389
:102C70009A4201D1C26822B9184650F8043B0B6051
:102C8000704700231846FAE7C368C2690133C3607E
:102C90004369134482694361934224BF436A436199
:102CA0000021FEF7E9BD000038B504460D46E36893
:102CB0003BB123691A1DA262E2691344E36200205A
:102CC00007E0237A33B929462046FEF7C5FD0028E0
:102CD000EDDA38BD6FF00100FBE700000369196011
:102CE000C268013AC260C2691344826903619342B7
:102CF00024BF436A036100238362036B03B1184757
:102D00007047000070B530230D460446114683F32A
:102D10001188866A2EB9FFF7C7FF10B186F31188B4
:102D200070BDA36A1D70A36AE26A01339342A36275
:102D300004D3E16920460439FFF7D0FF002080F377
:102D40001188EDE72DE9F84F04460D469046994667
:102D50004FF0300A8AF311880026B346A76A4FB9AC
:102D600049462046FFF7A0FF20B187F3118830467F
:102D7000BDE8F88FD4E90A073A1AA8EB060797428C
:102D800028BF1746402F1BD905F1400355F8042BE7
:102D900040F8042B9D42F9D1A36A4033A362403628
:102DA000D4E90A239A4204D3E16920460439FFF7A3
:102DB00095FF8BF311884645D9D28AF31188CDE768
:102DC00029463A46FDF746FFA36A3B443D44A362C9
:102DD0003E44E5E7D0E904239A4217D1C3689BB18A
:102DE000836A8BB1043B9B1A0ED01360C368013B0E
:102DF000C360C3691A44836902619A4224BF436A6B
:102E00000361002383620123184670470023FBE718
:102E100000F030B94FF08043586A70474FF080435C
:102E2000002258631A610222DA6070474FF0804333
:102E30000022DA60704700004FF08043586370470B
:102E4000FEE7000070B51B4B01630025044686B009
:102E5000586085620E4600F0BFF804F11003C4E923
:102E600004334FF0FF33C4E90635C4E90044A560DC
:102E7000E562FFF7CFFF2B460246C4E9082304F1C1
:102E800034010D4A256580232046FEF79BFC012373
:102E9000E0600A4A0375009272680192B268CDE957
:102EA0000223074B6846CDE90435FEF7B3FC06B0B4
:102EB00070BD00BF00260020BC360008C1360008E7
:102EC000412E0008024AD36A1843D062704700BFFF
:102ED000982300204B6843608B688360CB68C36095
:102EE0000B6943614B6903628B6943620B68036042
:102EF0007047000008B5264B26481A6940F2FF11BA
:102F00000A431A611A6922F4FF7222F001021A615F
:102F10001A691A6B0A431A631A6D0A431A651E4A24
:102F20001B6D1146FFF7D6FF02F11C0100F5806012
:102F3000FFF7D0FF02F1380100F58060FFF7CAFF0C
:102F400002F1540100F58060FFF7C4FF02F1700147
:102F500000F58060FFF7BEFF02F18C0100F5806094
:102F6000FFF7B8FF02F1A80100F58060FFF7B2FF9C
:102F700002F1C40100F58060FFF7ACFF02F1E0014F
:102F800000F58060FFF7A6FFBDE8084000F0EEB84E
:102F90000038024000000240C836000808B500F0C2
:102FA00059FAFEF7D3FBFFF793F8BDE80840FEF7A8
:102FB0005BBE000070470000EFF3098305494A6BD0
:102FC00022F001024A63683383F30988002383F304
:102FD0001188704700EF00E0302080F3118862B65E
:102FE0000C4B0D4AD96821F4E0610904090C0A432D
:102FF000DA60D3F8FC20094942F08072C3F8FC2063
:103000000A6842F001020A602022DA7783F822007F
:10301000704700BF00ED00E00003FA05001000E07B
:1030200010B5302383F311880E4B5B6813F40063F3
:1030300014D0F1EE103AEFF30984683C4FF080733E
:10304000E361094BDB6B236684F30988FEF752FBCF
:1030500010B1064BA36110BD054BFBE783F311884C
:10306000F9E700BF00ED00E000EF00E02F030008EB
:10307000320300080F4B1A6C42F001021A641A6EF8
:1030800042F001021A660C4A1B6E936843F001037A
:1030900093604FF0804353229A624FF0FF32DA621E
:1030A00000229A615A63DA605A6001225A611A60FA
:1030B000704700BF00380240002004E04FF080421B
:1030C00008B51169D3680B40D9B2C9439B07116198
:1030D00007D5302383F31188FEF74EFB002383F3DB
:1030E000118808BD1F4B1A696FEAC2526FEAD252AB
:1030F0001A611A69C2F308021A614FF0FF301A69A7
:103100005A69586100215A6959615A691A6A62F00C
:1031100080521A621A6A02F080521A621A6A5A6A55
:1031200058625A6A59625A6A1A6C42F080521A649A
:103130001A6E42F080521A661A6E0B4A106840F4FA
:1031400080701060186F00F44070B0F5007F1EBFF3
:103150004FF4803018671967536823F40073536085
:1031600000F054B90038024000700040334B4FF07B
:1031700080521A64324A4FF4404111601A6842F09A
:1031800001021A601A689107FCD59A6822F00302BE
:103190009A602A4B9A6812F00C02FBD1196801F070
:1031A000F90119609A601A6842F480321A601A684C
:1031B0009203FCD55A6F42F001025A671F4B5A6FB7
:1031C0009007FCD51F4A5A601A6842F080721A6054
:1031D0001B4A53685904FCD5184B1A689201FCD558
:1031E000194A9A60194B1A68194B9A42194B21D106
:1031F000194A1168194A91421CD140F205121A600D
:10320000144A136803F00F03052BFAD10B4B9A688D
:1032100042F002029A609A6802F00C02082AFAD17F
:103220005A6C42F480425A645A6E42F480425A66A2
:103230005B6E704740F20572E1E700BF0038024064
:10324000007000400854400700948838002004E0D3
:1032500011640020003C024000ED00E041C20F413B
:10326000074A08B5536903F00103536123B1054AC6
:1032700013680BB150689847BDE80840FFF7D0BE0F
:10328000003C0140E02D0020074A08B5536903F0D7
:103290000203536123B1054A93680BB1D068984784
:1032A000BDE80840FFF7BCBE003C0140E02D002017
:1032B000074A08B5536903F00403536123B1054A73
:1032C00013690BB150699847BDE80840FFF7A8BEE5
:1032D000003C0140E02D0020074A08B5536903F087
:1032E0000803536123B1054A93690BB1D06998472C
:1032F000BDE80840FFF794BE003C0140E02D0020EF
:10330000074A08B5536903F01003536123B1054A16
:10331000136A0BB1506A9847BDE80840FFF780BEBA
:10332000003C0140E02D0020164B10B55C6904F410
:1033300078725A61A30604D5134A936A0BB1D06A16
:103340009847600604D5104A136B0BB1506B984731
:10335000210604D50C4A936B0BB1D06B9847E2055C
:1033600004D5094A136C0BB1506C9847A30504D5DA
:10337000054A936C0BB1D06C9847BDE81040FFF73D
:103380004FBE00BF003C0140E02D0020194B10B59E
:103390005C6904F47C425A61620504D5164A136DD7
:1033A0000BB1506D9847230504D5134A936D0BB1AB
:1033B000D06D9847E00404D50F4A136E0BB1506EE0
:1033C0009847A10404D50C4A936E0BB1D06E984770
:1033D000620404D5084A136F0BB1506F9847230459
:1033E00004D5054A936F0BB1D06F9847BDE81040E4
:1033F000FFF716BE003C0140E02D002008B5FFF7A6
:103400005DFEBDE80840FFF70BBE0000062108B5D1
:103410000846FFF71DFB06210720FFF719FB0621D1
:103420000820FFF715FB06210920FFF711FB0621F5
:103430000A20FFF70DFB06211720FFF709FB0621E5
:103440002820FFF705FBBDE8084007211C20FFF7F7
:10345000FFBA000008B5FFF745FE00F00BF8FDF7D6
:1034600053FEFDF72BFDFFF7A5FDBDE80840FFF774
:10347000CFBC00000023054A19460133102BC2E9D6
:10348000001102F10802F8D1704700BFE02D0020C2
:10349000034611F8012B03F8012B002AF9D17047DC
:1034A00053544D3332463F3F3F0053544D33324621
:1034B0003430780053544D3332463432780053540C
:1034C0004D33324634343658580000000120330062
:1034D0000010410001105A0003105900071031007C
:1034E00000000000A034000813040000AA34000803
:1034F00019040000B434000821040000BE340008A0
:1035000000000000390E0008250E0008610E0008BA
:103510004D0E0008590E0008450E0008310E000837
:103520001D0E00086D0E00080000000001000000E4
:10353000000000006330000034350008F023002054
:10354000002600204172647550696C6F740025423A
:103550004F415244252D424C002553455249414C80
:1035600025000000020000000000000055100008C7
:10357000C110000840004000A02A0020B02A00200E
:103580000200000000000000030000000000000036
:10359000051100080000000010000000C02A0020F3
:1035A000000000000100000000000000682D002065
:1035B00001010200051C0008151B0008B11B0008D2
:1035C000951B000843000000CC35000809024300A9
:1035D000020100C0320904000001020201000524BA
:1035E0000010010524010001042402020524060044
:1035F00001070582030800FF09040100020A000018
:10360000000705010240000007058102400000009C
:1036100012000000183600081201100102000040DC
:1036200009124157000201020301000004030904CA
:1036300025424F41524425005370656564794265C7
:1036400065463430354D696E69003031323334357A
:1036500036373839414243444546000000400000B7
:103660000040000000400000004000000000010099
:103670000000020000000200000002000000020042
:103680000000020000000200000002000000000034
:103690004912000801150008AD150008400040005F
:1036A000C82D0020C82D002001000000D82D0020CA
:1036B0008000000040010000030000006D61696EA1
:1036C0000069646C650000000001812A00000000B0
:1036D000AAAAAAAA00010024FFFE00000000000020
:1036E00000A00A000000000100000000AAAAAAAA87
:1036F00000000001FFFF00000000000000000000CB
:103700000000001000000000AAAAAAAA00000010F1
:10371000FFFF0000000000000000000000000000AB
:1037200000000000AAAAAAAA00000000FFFF0000F3
:103730000000000000000000000000000000000089
:10374000AAAAAAAA00000000FFFF000000000000D3
:10375000000000000000000000000000AAAAAAAAC1
:1037600000000000FFFF000000000000000000005B
:103770000000000000000000AAAAAAAA00000000A1
:10378000FFFF00000000000000000000000000003B
:10379000000000000A00000000000000030000001C
:1037A0000000000000000000000000000000000019
:1037B0000000000000000000000000000000000009
:1037C00000000000000000006F0400000000000086
:1037D00000400F0000000000FF00960000000008FD
:1037E0000096000000000800040000002C360008CD
:1037F00000000000000000000000000000000000C9
:083800000000000000000000C0
:00000001FF
